:1000000073C004C272C38BC08AC089C088C087C055
:1000100086C085C084C083C082C081C080C01201F8
:10002000100102000008C016E105044601020001AB
:100030001003460075006E006B00550073006200EF
:100040005A0368006100660074006D0061006E0074
:100050006E00230073006F0066007400770061007B
:1000600072006500200028007700770077002E00DE
:10007000740075002D006300680065006D006E005F
:10008000690074007A002E00640065002F007E0075
:100090006800650068006100290004030904090282
:1000A0004300020100800509040000010202010072
:1000B000052400100104240206052406000105247D
:1000C0000103010705830308000A09040100020A6D
:1000D0000000000705010208000007058102080072
:1000E000003200000000000811241FBECFE5D1E05F
:1000F000DEBFCDBF10E0A0E6B0E0E2E8F9E003C06B
:10010000C89531960D92AE36B107D1F710E0AEE644
:10011000B0E001C01D92A93BB107E1F794C370CFD5
:10012000CF93B92FA82FC62F8091610084FF07C0FD
:1001300080918E0098E8892780938E0003C08AE51D
:1001400080936100EFE8F0E09C2F91509F3F19F001
:100150008D918193FACF6C2F8FE890E053D1CC5FD3
:10016000C0936100CF910895CF93B92FA82FC62FC8
:100170008091600084FF07C08091830098E8892700
:100180008093830003C08AE580936000E4E8F0E098
:100190009C2F91509F3F19F08D918193FACF6C2F36
:1001A00084E890E02FD1CC5FC0936000CF91089598
:1001B0001F93CF93DF9360919F0016160CF09FC0A2
:1001C00080919B00CFEAD0E0C81BD109635090E03A
:1001D00010E880919A00803120F48C2F9D2F32D32B
:1001E00088C08D3209F06EC04AE5409362006830E5
:1001F00009F07BC08881807609F051C021E830E0A9
:10020000909381008981882321F49093820092E069
:100210000FC0853021F48A818093A0004BC08630C6
:1002200039F510EC8B81813041F42EE130E092E120
:1002300030939E0020939D003DC0823021F42EE932
:1002400030E093E4F5CF8330A9F58A81882321F447
:100250002AE930E094E0ECCF813021F420E430E072
:10026000942FE6CF823031F520E330E090E1E0CF0B
:10027000883019F422EA30E008C0893021F48A81FC
:100280008093A20017C08A3011F491E0D1CF8B3057
:1002900089F48BE480938E00809383000BC08C2FB5
:1002A0009D2F8AD2982F8F3F29F4888187FF1CC009
:1002B0009E811AC08F818823C1F48E818917A8F48A
:1002C000982F13C080916E0087FD0FC08C2F9D2F3B
:1002D000B6D29FEF891731F4909363008EE180933B
:1002E000620002C0811190E010E010936E009093C4
:1002F000630080919F00181614F410929F00809163
:10030000620084FF51C0809163008F3F09F44CC0AC
:10031000682F893008F068E0861B809363001BE437
:1003200080916E0080FD13EC8F5F80936E00A9E7D3
:10033000B0E087FF1CC0E0919D00F0919E00962FD9
:10034000915086FF08C09F3F61F0C895802D8D9326
:1003500031969150F8CF9F3F21F081918D9391502C
:10036000FACFF0939E00E0939D0077270AC06623A2
:1003700031F08A2F9B2F50D2682F772702C060E080
:1003800070E0C62F693040F489E790E03BD09C2FA5
:100390009C5FC83028F401C09EE18FEF809363001A
:1003A00010937800909362009AE086B3867011F4FF
:1003B0009150D9F7992321F49093A000909399003C
:1003C000DF91CF911F9108958BB780648BBF8BE431
:1003D00080938E00809383000895A82FB92F80E02A
:1003E00090E041E050EA60956F5F58F42D9138EF4E
:1003F00082279795879510F0842795273F5FC8F34C
:10040000F3CF0895EADF8D939D930895CF93CFB7EF
:10041000CF93C395B29BE9F7B29B17C0B29B15C0AF
:10042000B29B13C0B29B11C0B29B0FC0B29B0DC058
:10043000C0919C00C395C0939C00C2B7D3BBD2B3FC
:10044000C2BBCD1BC1BBD3B3D1C00F92DF93C09150
:100450009B00DD27CD55DF4F012EB29B03C0DF91FE
:100460000F90DACF2F930F931F934F932FEF4F6F70
:1004700006B302FB20F95F933F9350E03BE065C079
:1004800016B30126502952FDC89556B3012702FB29
:1004900025F92F7306B3B1F05027102712FB26F968
:1004A00006B22230F0F000C016B3012702FB27F994
:1004B0000126502906B22430E8F54F77206816B39C
:1004C0000000F6CF50274F7D206206B2102F0000AB
:1004D00000C006B300265029102712FB26F906B2E9
:1004E000E2CF4F7B06B3206400C0DACF012650294B
:1004F000167006B269F14E7F2160012F16B328C035
:10050000002650294D7F06B22260102F29C00126F7
:1005100050294B7F06B22460012F2DC016B301264F
:100520005029477F2860000006B22EC04F7E06B3D8
:10053000206130C0422706B3499300265029102776
:1005400006B24FEF12FB20F9297F16B379F216702D
:1005500049F10126502906B2012702FB21F9237F28
:1005600006B371F2002650293150D0F006B21027A0
:1005700012FB22F9277E16B351F2012650290127DA
:1005800002FB06B223F92F7C49F2000006B31027C4
:1005900012FB24F90026502906B22F7939F270CFC8
:1005A00000271AC03B503195C31BD0400881033C43
:1005B00009F10B34F9F0209199001981110F1213F0
:1005C000EFCF4A81441F093651F10D3211F0013E3F
:1005D00039F74F7009F0042F0093A1003F915F910C
:1005E0004F911F910F912F91DF910F90CF91CFBF1E
:1005F000CF9118950091A100002381F310919F00E5
:100600001123D1F53430D2F130939F0000939A003A
:1006100010919B003BE0311B30939B002FC0009159
:100620009F0001304CF50AE54F7049F430916200AB
:1006300034FD25C000936200C8E7D0E024C04330F9
:1006400049F03091610034FD1AC000936100CEE89A
:10065000D0E019C03091600034FD11C000936000FB
:10066000C3E8D0E010C0052710E000C021C0052776
:1006700010E0C89508BB14C03AE501C032ED032E66
:10068000C0E0D0E032E017B31660C29A08B317BBDF
:1006900056E020E84FEF20FF052708BB2795179568
:1006A0001C3F28F700004552B0F720FF052727958B
:1006B00008BB17951C3FB8F629913A9561F7097F59
:1006C0001091A000110F08BBC250D04011F0109340
:1006D0009900046017B3197F402F497F54E05A9561
:1006E000F1F708BB17BB48BB79CF1F920F920FB62B
:1006F0000F9211248F939F9390917300B39910C020
:100700008FEF89BD947F909373008091740088234C
:1007100061F48AE08093750081E08093740005C0E5
:1007200080E389BD9B60909373009F918F910F90A0
:100730000FBE0F901F901895209174002223D9F1BD
:1007400090917500981B909375009923A4F59C5E79
:1007500090937500822F99278130910519F00A979F
:1007600061F01CC02F5F20937400809173008B7820
:1007700080937300B39B1FC00EC0B39905C08091D6
:10078000730084618093730080916F008093710087
:1007900081E08093720010927400089580916F0040
:1007A000869580936F00B39B03C0806880936F0031
:1007B0002F5F209374000895F92FE82F80819927E7
:1007C00080769070809729F52181822F9927803239
:1007D0009105CCF0823291051CF08497A4F405C0F9
:1007E000209376008FEF90E0089582819381892B8A
:1007F00031F0C498BC9A83E08093730004C0BC9825
:10080000C49A10927300808187FD03C088E08093B2
:10081000770080E090E00895282F392F80917600AE
:10082000813251F447E050E061EE70E0932F822F67
:100830009CD087E090E0089580E090E0089581E00A
:1008400090E008950895CFE5D1E0DEBFCDBF00E090
:1008500094B704BF479A88E10FB6F89481BD11BCE4
:100860000FBE93FF0EC086B3992786709070892BB8
:1008700041F080E48BBF80E385BFC49A789488956B
:10088000F89480E285BF8BE080BD83EC8ABD80E375
:1008900089BD82E083BF81E187BB28E028BB25BBFF
:1008A00080E68BBF88E190E00FB6F894A89581BDF3
:1008B0000FBE21BD89DD789486B39927867090702C
:1008C000892B09F0889510919C00C12FC01B31F431
:1008D00086B3992786709070892B09F4A89568DCF7
:1008E000CC2379F0012F91B39E50993F1CF481B72E
:1008F0008F5F81BF98301CF081B7815081BF8C2FF2
:100900001BDF8091610084FF10C0C0917200CC2376
:1009100021F48091770083FF08C06C2F81E790E07D
:10092000FFDB10927200C09377008091600084FF1B
:10093000C3CF80917000882389F4909173008091D7
:100940006C00981709F4B8CF90936C0068E084E6C7
:1009500090E00ADC81E080937000AECF62E08CE62C
:1009600090E002DC10927000A7CFE62FF72FA82F9F
:10097000B92F03C0C89531960D9241505040D0F721
:020980000895D8
:0E0982005A5A5AFFA120000000000200000097
:00000001FF
